:020000040800F2
:1000000040050020D90000082D1D0008C91900086E
:1000100000000000000000000000000000000000E0
:10002000000000000000000000000000771D000834
:100030000000000000000000751D0008791D000888
:10004000EB000008EB000008EB000008EB000008E4
:10005000EB000008EB000008EB000008EB000008D4
:1000600000000000EB000008EB000008EB000008B7
:10007000EB000008EB00000800000000EB000008A7
:1000800000000000EB00000800000000000000007D
:10009000EB00000800000000EB000008EB00000887
:1000A000EB000008EB000008EB00000885220008C8
:1000B000EB000008EB00000800000000000000005A
:1000C0000448854600F03AFB00480047912C0008A0
:1000D000C046C04640050020044880470448004709
:1000E000FEE7FEE7FEE7FEE7FEE7FEE7ED1D0008A0
:1000F000C100000830B50B46014600202022012433
:1001000009E00D46D5409D4205D31D469540491B4B
:100110002546954040191546521E002DF1DC30BD94
:10012000F0B51FB40646002082B005464024019178
:1001300000901BE0019922460F46304600F046FA37
:10014000049A059B801A994110D3104619462246FD
:1001500000F02CFA361A8F41019722460120002127
:10016000009F00F023FA38184D4100902046641E8D
:100170000028DFDC019B00982946324607B0F0BD1D
:10018000D2B201E00270401C491EFBD2704700222F
:10019000F6E710B513460A4604461946FFF7F0FF86
:1001A000204610BDF0B507460846584087B0C00F3E
:1001B000049048000E46590040084908BC1A88417E
:1001C00005D2384631461E4617460B4602465800B1
:1001D000400810434DD0300D039040055900400DAC
:1001E000490D0590401A0290402873DA1803012146
:1001F000000B09050843019004980092002806D0DE
:100200001146019A494200209041009101900298C4
:1002100040210A1A0199009800F0C8F905460C46D9
:100220006B4607CB00F0E3F9C0197141039A0E0D3C
:100230000023D71756401A467A40164344D0049AF2
:10024000002A2DD0029A012A039A15DC1205C01A41
:10025000914101263605001C7141D20F059ED2073F
:100260000093019202962A46234600F0E0F907B077
:10027000F0BD38463146FAE71605234A0F46B21854
:10028000C01AB74101210905001C4F4100187F41E8
:10029000114618187941E20F10436D19644113E0BB
:1002A000E2076D0815436408C2071443039A012648
:1002B0001205C01A91413605001C7141CE07400855
:1002C00030434908C01851412A46234600F0A2F99C
:1002D000CDE7FFE7049801224000C117121A00235E
:1002E0008B4104983146C417381AA141EEE730B467
:1002F0000124E407634030BC54E730B40124E40730
:10030000614030BC4EE700000000E0FFF0B51FB4D4
:1003100088B00B990998002448400999C00F4900FA
:1003200049080991C0070B990090490049080B91B1
:1003300009990898A64608431CD00B990A980843C7
:1003400018D0099801244000420D4800410D099839
:1003500024050003000B204309900B980003000BB9
:1003600020430B9050181C4940180022019014465D
:10037000104605E0002001460DB0F0BD032801DA6B
:10038000034600E003239C46C11A0AAE0AE05F0060
:1003900008ADED5B4F00F75B7D430027AA187C4159
:1003A000491C5B1E6145F2DD410004AB5A52210439
:1003B000120C0A43240C401C0828DFDB0198029031
:1003C0000099704601910090059B049A0799069840
:1003D00000F02DF9D0E700000DFCFFFFF0B50C4652
:1003E0005C4085B0E40FE40703944C0000266408E9
:1003F00059009446490802460296224321D062469B
:100400000A431ED06200570D4A000E032303550D08
:10041000012402462C492405781B1B0B360B40187F
:1004200023432643614600901C46501AB44103D32F
:100430000098401C009002E0921800985B41002850
:1004400003DA0020014605B0F0BD002001210905B6
:100450000746864611E064461D46141BB54106D387
:100460006546521BB341744607430C43A646CD076D
:1004700040084908284392185B4105460D43EAD1DC
:100480001046184313D06046194650407140084347
:1004900006D06046101AB34106D20122002306E0BE
:1004A00000220123DB0702E00122D243531000980F
:1004B00074460105381C6141029C039D0019694185
:1004C00000F0A8F8BFE70000FD03000070B54B0086
:1004D0005B0803430BD04B005C0D0026334665429E
:1004E000B341D417AD1AA34102DB0020014670BD11
:1004F00012053018514170BD0EB5C217C10F5040E2
:10050000CA0740180021054B0293019200910A4648
:100510000B4600F08CF803B000BD0000330400006F
:100520000EB505490291002100910A460B46019142
:1005300000F07DF803B000BD3304000070B5CD0FAE
:100540004A0009030123090B1B0519430B4BED0757
:100550000024520D9A4201DA002070BD074B34335B
:100560009A4203DC9A1A00F031F802E0044951186B
:1005700088402C43F1D0404270BD0000FF030000D2
:10058000CDFBFFFF10B5002904DB0124E407404246
:100590008C412146002B04DB1C460123DB07524221
:1005A000A3418B4200D1824210BD000010B5202A29
:1005B00004DB0146203A9140002010BD91402023E9
:1005C0009C1A0346E3401943904010BD10B5202A01
:1005D00004DB0846203AD040002110BD0B46D34032
:1005E000D0402024A21A91400843194610BD10B5EE
:1005F000202A06DBCB170846203A1041C1170B43CF
:1006000006E00B461341D0402024A21A9140084333
:10061000194610BD10B5002B08DA0024401C6141BA
:1006200092185B411A4301D14008400010BDF0B55B
:100630001FB482B005460C0003D0084601F03AFE14
:1006400002E001F037FE20300246009021462846A5
:10065000FFF7ACFF049B059A04460F46184311436D
:10066000084314D0184610431BD0009840210A1AA2
:1006700018460599FFF7AAFF05460E46009A059908
:100680000498FFF793FF084305D0012004E02046BB
:10069000394607B0F0BD0020C11705430E432C4377
:1006A000374300990E986305401A7905E40A002241
:1006B0000C43FD0A0A3002D500200146E9E7010596
:1006C000101969410C9C0D9D00196941FFF7A2FFAB
:1006D000DFE700004A0009030123090B1B0519434A
:1006E0000A4B10B5520D9A4202DA0020014610BDA5
:1006F000064B34339A4203DC9A1AFFF767FF10BDAA
:10070000034BD218FFF752FF10BD0000FF0300009B
:10071000CDFBFFFF10B5002904DB0124E4074042B4
:100720008C412146002B04DB1C460123DB0752428F
:10073000A341994200D1904210BD0000064C012512
:10074000064E05E0E36807CC2B430C3C9847103479
:10075000B442F7D3FFF7B8FC0C3000082C30000887
:100760000EB5FF200092012302900A460193EF216B
:10077000024800F0B7F90249C8700EBD34000020ED
:10078000000000200EB5FF2010230092019302907C
:100790000A460123EE21034800F04EFA0249C870D0
:1007A0000EBD00003400002000000020704770B52E
:1007B0000024014620314A79022A03D00421C16372
:1007C000012418E0026813680E25AB431360026829
:1007D00013685B085B001360436C1C22134001220A
:1007E00015469D40036C5D604A7100220A71816B61
:1007F000002900D08847204670BD70B5044600F03F
:10080000C7F80546601C00D0641C00F0C1F8401B0E
:10081000A042FAD370BD0000F8B500230124A2E085
:1008200027469F403A4070D04D68022D01D0122DCE
:1008300014D1DD08AD002D1800952D6A5E07AC4679
:10084000F50E0F26AE46AE406546B543AC460E6982
:100850007546AE4065462E43009D2E624D68012DC3
:1008600005D0022D03D0112D01D0122D16D185688F
:100870000326AC465D00AE46AE406546B543AC4689
:10088000CE687546AE4065462E43866046680D7953
:10089000BE43ED06ED0F9D403543456006685F00A1
:1008A0000325BD40AE46AE430D79B446AE07B60F44
:1008B000BE4065462E430660C6687546AE438D68E9
:1008C000BD403543C5604D68ED004BD5294D6E6B7D
:1008D00026436E639E08284DB6007519AC46AD6878
:1008E0009E07360F0F27B740BD4305273F07B84285
:1008F00001D1002715E0214FB84201D1012710E0B6
:100900001F4FB84202D102270BE02BE01D4FB84227
:1009100001D1032705E01C4FB84201D1052700E0B3
:100920000627B7402F436546AF60184D2E684F68C5
:100930009643FF0300D516432E606E684F689643BA
:10094000BF0300D516436E60AE684F689643FF0242
:1009500000D51643AE60EE684F689643BF0200D5DF
:100960001643EE605B1C0A681546DD4000D057E771
:10097000F8BD0000001002400000014000040050DB
:1009800000080050000C0050001C00500004014002
:1009900001480068704700002800002070B502463A
:1009A00040325378202B1CD11378012B19D001230E
:1009B000137024245470046825689D4325600468DE
:1009C00025681E03B5432560046825680D4325602E
:1009D00000680168194301602020507000201070E9
:1009E00070BD022070BD70B5024640325378202B96
:1009F0001BD11378012B18D00124147024235370B9
:100A000003681D68A5431D6005682B680F26360224
:100A1000B34309021943296000680168214301605A
:100A2000202050700020107070BD022070BD0000AA
:100A300070B5040006D025464035687800260028A9
:100A400002D005E0012070BD2E70204600F09AF91A
:100A500024206870206801684908490001600F215E
:100A60006068090688432168086121688A68012056
:100A7000C00382438A60E1680129A16808D021226D
:100A80009202114322689160E168022902D005E0D8
:100A90000143F7E701212268C902516021684A68D1
:100AA0000F4B1A434A602168CA688243CA60616971
:100AB00020690843A169090208432168C860216AC6
:100AC000E069084321680860206801680122114339
:100AD00001606664202068702663AE70002070BDDF
:100AE00000800002FFB5054604464035687883B0B3
:100AF000202875D10C98002814D00D98002811D00A
:100B0000287801286CD001202870FFF741FF0746A4
:100B1000012200901923D103204601F013F8002888
:100B200074D103E00120400260646FE0222068700D
:100B30004020A870002666640C9860620D9860855D
:100B400066630E980090019704A90EC9204600F034
:100B500085FF002801D02E7058E0618D3448FF29B0
:100B600005D9FF22228501231B06009006E0618D36
:100B700021850090208D0123C2B25B062046049996
:100B800000F0CCFF00970022042120460E9B00F0CD
:100B9000D9FF00283AD12068406A616A0870606A0B
:100BA000401C6062208D401E81B22185608D401EF8
:100BB0006085608D00281FD000291DD1009700227C
:100BC000802120460E9B00F0BDFF00281ED1608DC5
:100BD000FF2806D9FF22228501231B06009607E085
:100BE00024E0608D20850096208D0123C2B25B0633
:100BF0002046049900F092FF608D0028C2D13A4649
:100C000020460E9900F0C5FF002802D0012007B051
:100C1000F0BD20682021C16120684268054B1A4060
:100C200042606970AE702E700020F0E70220EEE79F
:100C30000024008000E800FEFFB50546044640356C
:100C4000687883B0202872D10C98002814D00D98B1
:100C5000002811D02878012869D001202870FFF7DA
:100C600097FE0746012200901923D103204600F089
:100C700069FF002871D103E00120400260646CE04C
:100C8000212068704020A870002666640C9860627D
:100C90000D98608566630E980090019704A90EC9AF
:100CA000204600F00BFF002801D02E7055E0608D2B
:100CB000FF2805D9FF22228501231B06009606E0A6
:100CC000608D20850096208D0123C2B25B062046F0
:100CD000049900F023FF3A4620460E9900F07FFF6A
:100CE00000283AD1606A216800788862606A401CF6
:100CF0006062608D401E6085208D401E80B2208520
:100D0000618D00291FD000281DD10097002280216D
:100D100020460E9B00F016FF00281ED1608DFF2894
:100D200006D9FF22228501231B06009607E024E056
:100D3000608D20850096208D0123C2B25B0620467F
:100D4000049900F0EBFE608D0028C4D13A4620469D
:100D50000E9900F01EFF002802D0012007B0F0BD60
:100D600020682021C16120684268054B1A4042601A
:100D70006970AE702E700020F0E70220EEE70000F0
:100D800000E800FE10B586B0044614216846FFF75F
:100D9000FEF91149206888421BD1104CE16A0220FB
:100DA0000143E162E16A0140032005918002009065
:100DB000122001900120029003200390062004904D
:100DC00069460748FFF728FDA06B01218905084304
:100DD000A06306B010BD00000058004000100240A3
:100DE0000004005002480168491C0160704700007F
:100DF0002800002010B50848002401684022114353
:100E00000160204600F00AF8002801D0012401E02A
:100E100000F01CF8204610BD0020024070B50546C9
:100E200009487D210024C9000068FFF763F900F03C
:100E3000F9FB002801D0012404E000222946501EBD
:100E400000F01AF8204670BD2C0000200448416BC9
:100E5000012211434163816B020411438163704796
:100E600000100240C106C90E0120884001490860F7
:100E70007047000000E100E010B500F059FF10BD20
:100E8000F8B504460078544D800672D5524E0027BE
:100E9000403EB06BC00004D4B06BA9050843B063FA
:100EA00001274E480168C90511D401688215114314
:100EB0000160FFF76DFD009005E0FFF769FD009907
:100EC000401A642837D845480068C005F5D532680F
:100ED0000321090560680A400140914208D081035E
:100EE000890F032904D13168890301D50120F8BD98
:100EF0002A69032109040A4022D0084090421FD0E9
:100F0000207880061CD528692A6988430121C904F4
:100F10000A432A612A698A432A612861C0050FD5DC
:100F2000FFF736FD009008E0FFF732FD0099411A07
:100F30002B48814201D90320F8BD28698005F3D5EB
:100F400061688803800F032805D132680005824359
:100F500001400A433260286903226168120411408B
:100F600008432861002F04D0B16B012000078143A2
:100F7000B1632078C00705D0E868A16880088000C8
:100F80000843E8602078800705D5E8680C2188438D
:100F9000E1680843E8602078400706D5E868032147
:100FA0008902884321690843E8602078000706D554
:100FB000E86803210903884361690843E8602078F1
:100FC000000606D5E868032189048843A16908431F
:100FD000E8600020F8BD00004010024000700040B2
:100FE00088130000F8B50E4605007DD05348006810
:100FF000C007C00FB0420AD25048016849084900F2
:10100000314301600068C007C00FB04271D1287839
:101010004B4C800705D5E068F0218843A968084358
:10102000E0602878C00752D06868022817D00328EB
:1010300018D02168012818D08905002959DAE168FB
:10104000890889000143E160FFF7A2FC696807464F
:10105000022912D003291CD0012926D033E02168AF
:101060008903EAE721688901E7E74907E5E7FFF730
:101070008FFCC11B3348814223D8E0680007800FF2
:101080000228F4D123E0FFF783FCC11B2D488142E5
:1010900017D8E0680007800F0328F4D117E0FFF7A6
:1010A00077FCC11B274881420BD8E0680007800FFE
:1010B0000128F4D10BE0FFF76BFCC11B21488142F2
:1010C00001D90320F8BDE0680007800FF3D11B4869
:1010D0000168C907C90FB1420DD901684908490023
:1010E00031430160006800E003E0C007C00FB04278
:1010F00001D00120F8BD2878400706D5E068072117
:1011000009028843E9680843E0602878000707D5AA
:10111000E0680721C90288432969C9000843E060E3
:1011200000F036F8E168084A0906090F515CC8402A
:10113000064908600020FFF771FEF8BD002002405C
:101140000010024088130000E82F00082C00002047
:10115000044805490068C968044A4905490F515CBB
:10116000C84070472C0000200010024001300008E9
:10117000044805490068C968044A8904490F515C5C
:10118000C84070472C0000200010024001300008C9
:1011900010B5184AD1680C20084004280BD0082844
:1011A00010D00C2810D050680004410F0120C0035B
:1011B000491C884010BD1068C00601D50E4810BDFE
:1011C0000E4810BD0E4810BD88020E4B000F185C73
:1011D0000902D368890F491CDB0301D5084A05E0E1
:1011E0001268D20601D5044A00E0044A5043FEF7D3
:1011F00081FF10BD0010024000093D000024F400F2
:1012000000127A00F82F0008FEB505007ED0FE4CD3
:10121000E7680C20E66807400120000406402878B3
:10122000C00747D0082F05D00C2F0AD10120000499
:10123000864206D1206880033CD568680028E5D046
:1012400038E0012069680004814203D1216801432C
:10125000216011E0052301221B04920499422168B8
:1012600002D111432160F1E78143216021680140EF
:101270000091206890432060686800280DD0FFF737
:1012800087FB009005E0FFF783FB0099401A642874
:101290007AD820688003F6D50CE0FFF779FB009040
:1012A00005E0FFF775FB0099401A6428F0D8206824
:1012B0008003F6D42878800755D50923E868042FE1
:1012C0000DD00C2F01D1002E09D000283BD0216871
:1012D000994301432160FFF75BFB064627E0216845
:1012E000490701D5002891D061681F22120291435D
:1012F0002A69120211436160216899430143216008
:10130000FFF746FFE16809060A0F00E079E1BF49EF
:10131000895CC840BE4908600020FFF77FFD0028B7
:1013200072D120E0FFF734FB801B0228B0D8206880
:101330004007F7D560681F2109028843296909021F
:10134000084360600FE02068400840002060FFF71D
:101350001FFB064604E0FFF71BFB801B022897D803
:1013600020684007F7D42878C0065FD5002F0CD03E
:10137000A869002849D02068FF2101310843206076
:10138000FFF706FB06462DE0C0E02068800502D589
:10139000A8690028A7D06068072149038843296A03
:1013A000084360606068297F0002000A090608435C
:1013B0006060286A410B0120C003491C8840E16835
:1013C00009060A0F9149895CC840914908600020CC
:1013D000FFF724FD002817D128E0FFF7D9FA801B7A
:1013E0000228A3D820688005F7D560680721490343
:1013F0008843296A084360606068297F0002000A08
:1014000009060843606011E0E1E02168FF20013037
:1014100081432160FFF7BCFA064604E0FFF7B8FA03
:10142000801B022872D820688005F7D42878794E6E
:10143000000724D568690028306910D001210843CD
:101440003061FFF7A5FA009005E0FFF7A1FA0099D7
:10145000401A02285AD830698007F6D50FE04008B4
:1014600040003061FFF794FA009005E0FFF790FA32
:101470000099401A022849D830698007F6D42878A4
:10148000400765D500200290A06BC00006D4A06B79
:10149000012109070843A063012002905E4801680A
:1014A000C90511D40168821511430160FFF770FA74
:1014B000009005E0FFF76CFA0099401A642825D8DF
:1014C00055480068C005F5D5FF20AA680130824262
:1014D00003D131690143316111E001218902002A00
:1014E00007D005231B029A4203D132690A433261B5
:1014F000EFE7326982433261306988433061A8681E
:1015000000280FD0FFF744FA009007E05EE0FFF7F5
:101510003FFA0099411A4148814257D83069800505
:10152000F5D50DE0FFF734FA009006E0FFF730FA4A
:101530000099411A3948814248D830698005F5D46C
:101540000298002804D0A06B012109078843A063FA
:10155000686A002864D00C2F3ED001263606022887
:10156000206805D0B0432060FFF712FA05462FE04F
:10157000B0432060FFF70CFA074604E0FFF708FAD3
:10158000C01B022822D820688001F7D4E96AA86A23
:10159000E2680843296BFD231B049A431143084367
:1015A000E060206830432060FFF7F2F9054604E070
:1015B000FFF7EEF9401B022808D820688001F7D514
:1015C0002EE0FFF7E5F9401B022801D90320FEBDFC
:1015D00020688001F5D423E00128F8D0E0680121DB
:1015E0000904AA6A014091420BD10F218904EA6AD9
:1015F0000140914205D1032189050840296B8842A9
:101600000ED00120FEBD000000100240E82F0008AF
:101610002C000020401002400070004088130000A1
:101620000020EFE7094910B5401E884201D901208A
:1016300010BD074C60610321081F00F079FB0020FA
:10164000A06107202061002010BD0000FFFFFF0007
:1016500000E000E0F0B502462032137E012B15D0E9
:10166000012717760223537605686C68AB687026ED
:10167000B4430E68496826438024A34319436E602F
:1016800000688160577600201076F0BD0220F0BD22
:1016900070B5040005D025462035687E002802D0AC
:1016A00006E0012070BD00202876204600F00AF8F0
:1016B00002206876211D206800F0C2FB01206876B8
:1016C000002070BD00680449884204D10348816B42
:1016D0001022114381637047001000400010024047
:1016E00070477047F8B502680446D069116893687E
:1016F00005072D0F5BD0DD07ED0FFF2621360E40CD
:101700002E4367D0C60706D0CE0504D50126166243
:10171000E26F3243E267870702220426002F06DACF
:10172000DF0704D027683A62E76F3743E767470768
:1017300006D5DB0704D023681E62E36F1343E3671B
:10174000020709D520220A402A4305D0236808222F
:101750001A62E36F1343E367E26F002A2FD080061B
:1017600006D5880604D5216E002901D02046884779
:10177000E06F21688968490601D4000724D5204616
:1017800000F02AFC20688168490619D5816840224A
:1017900091438160E06E002812D020498163E06EA1
:1017A000FFF705F800280AD0E06E816B06E0850699
:1017B00010D58D060ED5216E1CE020468847F8BD59
:1017C0002046FFF78EFFF8BD2046FFF78AFF002076
:1017D000E067F8BDC50208D55B0206D5012000050B
:1017E00010622046FFF77CFFF8BD030605D50B0607
:1017F00003D5616E0029E0D1F8BD4006FCD548064E
:10180000FAD51368204640218B431360202161677D
:101810000021616600F0D7F8F8BD0000C51F000880
:1018200010B5040003D0606F002802D007E001204B
:1018300010BD002170200155204600F027F824201B
:10184000606720680168490849000160204600F08F
:10185000D3FB0128ECD0606A002802D0204600F0BB
:101860001BFB206841680922D20291434160206835
:1018700081682A2291438160206801680122114316
:101880000160204600F06EFB10BD000010B586B070
:10189000044614216846FEF77AFC15492068884200
:1018A00024D11448416B0122920311434163C16A60
:1018B00001221143C162C06A6946104005900320AD
:1018C000400200900220019000200290032003902B
:1018D0000420049005200007FEF79EFF0022114619
:1018E0001B20FFF7C9FA1B20FFF7BCFA06B010BD9A
:1018F0000038014000100240FFB50446406F83B03D
:1019000017460D4620285CD1002D0AD0002F08D0A4
:10191000A168C001814207D12069002804D1E807ED
:1019200002D0012007B0F0BD204660300290007C5C
:10193000012846D00298012101740020E06721208F
:101940006067FFF725F82646403601903782778298
:101950000120A1680003814202D12069002802D041
:101960002F46002511E000270FE0002280212046AD
:1019700000F056FC002815D1002F15D021683878CA
:1019800088627F1C708A401E7082708A019B0028CA
:1019900006980090E9D100224021204600F040FC4A
:1019A000002808D00320BDE728882168C005C00DA5
:1019B0008862AD1CE6E72020606702990020087469
:1019C000B0E70220AEE77047FEE701688A69D243BC
:1019D000920701D400228A6200688169C943C9075D
:1019E00003D081690122114381617047F7B5044634
:1019F00000680E468069C043C0062BD420272546C8
:101A0000403520688069C043800612D5701CF8D02C
:101A1000FEF7BEFF0299401AB04201D8002EF0D165
:101A2000606C384360646F700020A87028700120DB
:101A3000FEBD21681020C8612068C7612046FFF7FD
:101A4000C4FF20684168044A11404160606C042171
:101A50000843E7E70020FEBD00E800FEF8B50446B5
:101A6000164615481D46DAB20090079F002320460F
:101A700000F054F83A462046069900F0B0F80028E5
:101A800018D12846F5B2012809D02168300A8862A9
:101A90003A462046069900F0A2F800280AD12068AC
:101AA00085620097002240212046069B00F04AF8FC
:101AB000002800D00120F8BD00200080F8B50446C1
:101AC000164615481D46DAB2C3020090079F20460D
:101AD00000F024F83A462046069900F080F80028E5
:101AE00018D12846F5B2012809D02168300A886249
:101AF0003A462046069900F072F800280AD120687C
:101B000085620097002280212046069B00F01AF88B
:101B1000002800D00120F8BD00200080F0B5066844
:101B2000059C7568064F600D384385438805800D18
:101B3000110408431843204305437560F0BD0000BD
:101B4000FF63FF03F8B51D4617460E46044609E03D
:101B5000681C07D0FEF71CFF0699401AA8420BD854
:101B6000002D09D020688169304688430FD00020BD
:101B7000B842EDD00020F8BD616C202001436164C3
:101B8000403460700020A07020700120F8BD01205A
:101B9000EEE770B516460D4604460FE0324629467C
:101BA0002046FFF723FF002801D0012070BDFEF77B
:101BB000EFFE801BA84208D8002D06D0206880695F
:101BC000C0438006EAD4002070BD616C2020014330
:101BD0006164403460700020A0702070E5E770B54B
:101BE00016460D46044611E0324629462046FFF7C8
:101BF000FDFE002801D0012070BD681C06D0FEF754
:101C0000C7FE801BA84208D8002D06D02068806936
:101C1000C0438007E8D4002070BD616C20200143E0
:101C20006164403460700020A0702070E3E7000021
:101C300008B50848C26A02210A43C262C26A0A4061
:101C40000092C16A01221143C162C06A1040009033
:101C500008BD00000010024010B514481249016090
:101C6000E121C90041600021816001614161816120
:101C70000122C161C2600162FEF7DAFE002801D0D4
:101C8000FEF794FD00210948FEF788FE002801D0E8
:101C9000FEF78CFD00210548FEF7A5FE002801D0C7
:101CA000FEF784FD10BD0000005800403400002005
:101CB0001CB500240E4800940C49019401600721D2
:101CC0008460416001214461C160FFF7E1FC0028AC
:101CD00001D0FEF76BFD0094694605480194FFF7BB
:101CE000B9FC002801D0FEF761FD1CBD00100040CA
:101CF0008000002010B50C480A490160E12149022A
:101D0000416000218160C16001618161C1610C227B
:101D1000016242614162FFF783FD002801D0FEF7B6
:101D200045FD10BD00380140BC0000207047000098
:101D30008307FF22DB0E9A408907090E994000288D
:101D40000BDA0007000F0838830808489B001818B2
:101D5000C36993430B43C3617047830804489B00E6
:101D60001B181868904308431860704700ED00E0A6
:101D700000E400E07047704710B5FFF733F810BD7E
:101D800030B599B034216846FEF701FA14210DA848
:101D9000FEF7FDF91C2112A8FEF7F9F912480168B7
:101DA0000322D2029143C2148918016002200090DC
:101DB0000024102009940125049003956846FFF73C
:101DC00023FA0F200D9080200F900E951094002183
:101DD00011940DA8FFF706F912A812951494FFF7B5
:101DE0004FF819B030BD0000007000401048016885
:101DF000821511430160C1680E4A1140C16001683B
:101E00000D4A1140016081684908490081600168FC
:101E10000122920491430160C168FD2212049143A2
:101E2000C160002101610549C0038860704700005E
:101E3000001002400C40FF88F6FFF6FE00ED00E0C7
:101E400070B5026801239B07114C124D984203D0D4
:101E5000A04201D0A84203D17026B2434E6832435B
:101E6000984203D0A04201D0A84204D103231B0210
:101E70009A43CB681A4380239A430B691A43026042
:101E80008A68C262096881620121416170BD0000F7
:101E9000000801400014014010B5818CC90707D02B
:101EA00001684A6801235B049A43836A1A434A60C3
:101EB000818C890707D501684A6801231B049A436E
:101EC000C36A1A434A60818C490707D501684A688A
:101ED00001239B049A43036B1A434A60818C0907D0
:101EE00007D501684A680123DB039A43436B1A4311
:101EF0004A60818CC90607D50268916801231B03DB
:101F00009943836B19439160818C890607D50168D9
:101F10008A6801235B039A43C36B1A438A60818CEE
:101F2000490612D503685A6801210905046C8A43E1
:101F300022435A60026C8A4207D102685168032327
:101F40005B059943436C19435160818C090607D5A1
:101F500001684A680123DB04806C9A4302434A60AB
:101F600010BD0000F8B500260446C667FEF710FD58
:101F7000054620680068124F000709D501212B464D
:101F8000002249052046009700F04AF900280DD1AB
:101F90002068006840070BD501212B4600228905E7
:101FA0002046009700F03CF9002801D00320F8BD3E
:101FB00020206067A067603426740020F8BD000010
:101FC000FFFFFF0110B5806A0022014640314A83BD
:101FD0004A82FFF786FB10BD01680A68FF232133A0
:101FE0009A430A6001688A68520852008A60202178
:101FF0008167002101667047F8B504462669A2682A
:10200000E76932436669102000253E432368324366
:1020100078491E68784F3E4016431E6023685A6810
:1020200003263603B243E66832435A602368A26946
:102030008B4201D0266A32439E680B273F02BE4383
:1020400016439E606D4E23686D4AB3420CD1D26830
:102050009207920F06D0012A38D0022A34D0032AE0
:1020600020D11EE001201DE0664EB3420AD1D268A5
:102070000C26324026D0042A28D0082A24D00C2A44
:1020800010D10EE08B420DD1D66803229202164089
:1020900018D001229202B61A18D0B61A14D096425D
:1020A00000D10820564A0126403A574FF6038B428A
:1020B00036D100280CD002280DD0042812D00828D0
:1020C0001FD11CE00020EDE70220EBE70420E9E748
:1020D000FFF73EF808E01068C00601D5384605E075
:1020E0004A4803E0FFF754F8002873D062685100B3
:1020F0005118814205D81103814202D303E03046D2
:10210000F4E7012566E0010E0602500800233018AE
:102110005941FEF705F803210902411A3C4A55E0EE
:10212000E169B14232D1030000F0DBF809070A0D82
:1021300006250606062B0600E3E7FFF709F81CE074
:10214000FFF716F819E010686168C00602D5480864
:10215000304A01E0304A48088018FDF7CBFF80B2D2
:1021600001462E4A10399142CBD8511C014000073C
:10217000400F08432CE0FFF70BF8616840004A0865
:10218000EAE76168012248081204E5E7030000F06D
:10219000A8F809070A0D06260606062C0600B0E771
:1021A000FEF7D6FF1DE0FEF7E3FF1AE01068616856
:1021B000C00602D54808C01902E014484A081018A1
:1021C000FDF798FF80B20146144A1039914298D821
:1021D0002168C8600020206660662846F8BDFEF7CA
:1021E000D7FF61684A088018EAE7616848088019E3
:1021F000E6E7000000480040F369FFEF00380140C7
:10220000401002400044004000093D000024F4005A
:10221000FFFC0F0000127A000048E801EFFF000009
:10222000FFB581B017460E4604460A9D09E0681CBA
:1022300007D0FEF7ADFB0499401AA8420CD8002D38
:102240000AD02068C1693046884318D00020B842BF
:10225000EDD0002005B0F0BD20680168FF22A1325A
:10226000914301602068816849084900816020200D
:102270006067A0670020603420740320EAE7012033
:10228000E5E7000010B50248FFF72CFA10BD00008A
:10229000BC0000200FB410B503A9044B044A0298F7
:1022A00000F0F6F810BC08BC04B01847752C000804
:1022B000300000202021020C01D010211046020A1B
:1022C00001D010460839020901D01046091F8208C2
:1022D00001D01046891E420801D0881E7047081A96
:1022E000704730B47446641E2578641CAB4200D23B
:1022F0001D46635D5B00E31830BC184702E008C868
:10230000121F08C1002AFAD170477047002001E06F
:1023100001C1121F002AFBD170470000F0B51FB4A5
:1023200086B00998089A030D0021024314D0514841
:10233000514A1818504305141198012810981AD0C2
:10234000281A401C00264D4F4D49009601910490DB
:10235000002812DA444211E01198012449A301280F
:1023600001D11098C1430698119A84600360C2603D
:1023700041600BB0F0BD4042E4E704462105002077
:102380003F4A001C51410391029012E0E00707D040
:1023900032463B4601990098FDF7B8FF0191009045
:1023A00032463B4610461946FDF7B0FF06460F463B
:1023B0006410002CEAD10498039B0028029A099922
:1023C000089806DAFDF7A2FF019B009AFDF79EFF31
:1023D00005E0FEF703F8019B009AFDF7FFFF0446B6
:1023E0000E460022284BFEF795F903D80020C04383
:1023F000014607E00022254B20463146FDF7D2FE7C
:10240000FEF768F9102409E0002C0ADB0A220023F9
:10241000FDF786FE079B30321A55641E02460A43BA
:10242000F2D11122641C079B121B1C19119B012B5A
:1024300003D0012308430ED10AE0084304D0112041
:1024400010900020119077E71098151A6D1E0BE080
:102450001098824202DD00236D1C03E0824201DA03
:1024600000236D1E002BEED0069811998260C1608A
:1024700030C07EE701FCFFFF104D0000000014405B
:102480000000F03F300000000000F0430000E03F9B
:10249000FFB597B0064600251BE2252876D100241B
:1024A0002746F749049400E00443761C3278012063
:1024B000203A90400842F7D130782A280ED00222E4
:1024C000307801463039092916D804990A2359432E
:1024D000303940181443761C0490F1E7189802C86C
:1024E00004911890002904DA012040030443484273
:1024F000049002200443761C30782E2814D1042046
:1025000004437078761C2A2809D11898761C80C854
:10251000189009E00A214F43303FC719761C3078E4
:10252000014630390929F5D930786C2810D006DCFD
:102530004C281AD068280ED06A2817D104E07428D5
:1025400013D07A2812D110E00120400504430CE09A
:102550000121090501E0032109050C43717881423D
:1025600003D1012000052418761C761C30786628DB
:102570000BD013DC58287DD009DC00287BD04528FF
:10258000F6D04628F4D047281AD1A9E118E06328EC
:1025900035D0642870D0652812D1A1E170286CD0A4
:1025A00008DC6728F1D069287DD06E280DD06F280F
:1025B00006D1BCE073282ED0752873D0782859D066
:1025C0001A9A199990476D1C82E16002400F022807
:1025D00009D003280DD00428189801680DD00D608B
:1025E000001D189074E11898EA1701680D604A60A0
:1025F000F6E7189801680D80F2E70D70F0E718987B
:102600006A4601781172001D18900020507202A8CD
:102610000090012005E0189802C818900020009151
:10262000C04361070ED5002101E00199491C0191C9
:10263000B94213DA8142F8DB019A0099895C0029DA
:10264000F3D10BE0002101E00199491C0191814285
:10265000FADB019A0099895C0029F5D10199049867
:102660001A9B471A21463846199A00F099FA4019E0
:10267000019903E051E030E115E050E0451807E032
:10268000009800990078491C00911A9A199990476E
:102690000198401E0190401CF2D1214638461A9BF9
:1026A000199A12E137E00A2000210090019160029E
:1026B000410F022907D0189A01CA1892C2179446EE
:1026C000032908D00AE01898C01DC108C90005C92F
:1026D0001891944607E000B2C2179446042902D12B
:1026E00040B2C1178C4600226146944506DA0A467C
:1026F0000021404291418C462D2102E0210504D564
:102700002B216A461173012103E0E10701D020214A
:10271000F7E7029156E00A200AE0102008E01020B6
:1027200000900021042004430191082703E00820C1
:102730000021019100906002410F022907D0189AF0
:1027400001CA189200229446032908D008E018987C
:10275000C01DC108C90005C91891944603E080B2A4
:10276000042900D1C0B20021029121072AD5317875
:102770000D91702906D0009A1021019B4A401A43FE
:1027800005D00EE040216A461173012108E0614640
:10279000014306D030216A4611730D99517302210D
:1027A0000291009A0821019B4A401A430AD16146CE
:1027B000014301D1610705D530216A46117301211A
:1027C0007F1E02913178582904D02EA10E910DA9B7
:1027D0000D910DE030A1F9E76146019B009AFDF7EC
:1027E0009FFC0E9B8C469B5C0D9A521E0D921370A3
:1027F00061460143F0D10D9805A9081A20300190D7
:10280000600703D501200004844300E001270198FC
:10281000874201DD381A00E000200199009041183C
:10282000029809180498401A0490E00306D421463F
:102830001A9B199A049800F0B3F94519002706E08D
:1028400003A81A9AC05D199990476D1C7F1C0298C5
:102850008742F5DBE0030CD521461A9B199A0498B0
:1028600000F09EF9451904E01A9A30201999904712
:102870006D1C0099481E00900029F5DC1FE0000047
:102880000928010030313233343536373839616246
:10289000636465660000000030313233343536370A
:1028A0003839414243444546000000000D980D99D7
:1028B0000078491C0D911A9A199990476D1C01993D
:1028C000481E01900029F1DC4DE100F059F945194D
:1028D000761C3078002800D0DFE528461BB0F0BD1C
:1028E000600700D406271898C01DC108C9004868B1
:1028F0000A680831C30FDB071891190001D09CA1A9
:1029000008E0210501D59BA104E0E10701D09AA1CF
:1029100000E09AA14300109130785B0865280CD044
:1029200006DC452809D046281DD0472841D141E082
:10293000662818D067283CD13CE00021112F01DB2C
:10294000112000E0781C0191009008A911A8FFF760
:10295000E5FC139905910021119A15927F1C12989C
:102960000197009150E00120C007039001200190E1
:1029700008A9009711A8FFF7D1FC139A14990592A2
:102980000022119B009212981593059A019200293A
:1029900001D0104602E0791C40180190381A01D588
:1029A000019804E04042401E0090781C0190C01B3A
:1029B000029043E0012F00DA01270021112F01DDF1
:1029C000112000E038460191009008A911A8FFF7F6
:1029D000A5FC13990591119A002112981592009166
:1029E000019721070CD40599B94201DB019900E058
:1029F0000191012904DD159A491E515C302906D048
:102A0000B84201DA011D05DA0121029115E00199B0
:102A1000491EEDE7002805DC009941180091019955
:102A2000091A03E0019A411C914200DD01910099CD
:102A3000401A401C02900120C0070390200706D4D2
:102A400002990198814202DB0020C04302900020DD
:102A50006946C87707AF012103980337C907884241
:102A600024D0022011902B201290039800280CDA19
:102A7000404203902D20129007E00A210398FDF7B1
:102A800039FB30317F1E039039701199481E119027
:102A90000029F2DC03980028EFD1791E1298087003
:102AA0003078202108404530BF1E387006A8C01B72
:102AB000C01D039010980078002800D001200199D3
:102AC00041180298C0170918039809180498401A69
:102AD000401E0490E00306D421461A9B199A0498DC
:102AE00000F05EF8451910980078002803D01A9A73
:102AF000199990476D1CE00324D521461A9B199A19
:102B0000049800F04DF845191CE00098002807DBF8
:102B100000990598884203DD1598405C199901E0F9
:102B2000199930201A9A904700986D1C401C00900B
:102B30000298401E0290002804D11A9A2E2019995A
:102B400090476D1C0199481E01900029DDDC05E0CD
:102B500038781A9A7F1C199990476D1C0399481E62
:102B600003900029F4DC21461A9B199A0498ACE6DC
:102B70002D0000002B0000002000000000000000DD
:102B8000F8B5044600251E461746880404D405E01F
:102B900039462020B0476D1C641EF9D52846F8BD83
:102BA000FFB50446002581B01E46C80301D5302775
:102BB00000E02027880404D505E038460399B04793
:102BC0006D1C641EF9D5284605B0F0BD70B50446ED
:102BD0000146084A0848FDF7C3FD064D641C2E78DF
:102BE000A1B22A460448FDF7BBFD28780002304315
:102BF00000B270BD040000203400002070B50C4A03
:102C0000F7210C48FDF7ACFD094CF8212678224647
:102C10000848FDF7A5FD25782246F9210548FDF76E
:102C20009FFD217830032A0110430909084370BD34
:102C3000040000203400002070B50C4AFA210C4832
:102C4000FDF78EFD094CFB21267822460848FDF74A
:102C500087FD25782246FC210548FDF781FD217876
:102C600030032A0110430909084370BD0400002005
:102C70003400002001B5044B012269460348FEF7E9
:102C80003BFE009808BD0000FFFF0000BC000020D4
:102C9000F0B58BB0FEF7AEF8FFF772F8FEF7C8FF9D
:102CA000FFF728F8FFF704F8FEF7D6FFC04AE02147
:102CB000C048FDF767FDBE4AF421521CBD48FDF730
:102CC00061FDBB4AF521921CBA48FDF75BFD8820E7
:102CD000FFF77CFFB64CE0808A20FFF777FF20816A
:102CE0008C20FFF773FF60818E20FFF76FFFA081BC
:102CF0009020FFF76BFFE0819220FFF767FF2082B3
:102D00009420FFF763FF60829620FFF75FFFA082A9
:102D10009820FFF75BFFE0829A20FFF757FF2083A0
:102D20009C20FFF753FF60839E20FFF74FFFA08397
:102D3000FFF782FF9E4C6062FFF760FF20622089F0
:102D4000FDF7EEFB09910890E088FDF7E9FB092209
:102D50000746D2430591FDF7B9FB05460191606A2C
:102D6000FDF7DEFB0D220646D2430391FDF7AEFBD5
:102D70002A46019BFDF7BBFA099B089AFDF7C6FAA4
:102D800000900D466089FDF7CBFB079106900C2261
:102D90003846D2430599FDF799FB07460591102265
:102DA0003046D2430399FDF791FB3A46059BFDF768
:102DB0009EFA02460B46FDF7A9FA079B069AFDF715
:102DC000A5FA02460B4629460098FDF7EBF90546A1
:102DD0000191FDF7B3FBFDF78FFB06460F46284632
:102DE0000022754B0199FDF7F9FA02460B4673A0D4
:102DF000FFF750FA0022D24330463946FDF766FB12
:102E00000022714BFDF773FA05460E46E08AFDF786
:102E100087FB07462A463346059110461946FDF7BB
:102E200075FA3A46059BFDF771FA0E22D243FDF77B
:102E30004DFB02900F46A08AFDF772FB2A463346EF
:102E4000FDF764FA0122FDF741FB3B46029AFDF7CC
:102E5000A9F903910290608AFDF762FB1022FDF749
:102E600035FB074601220491D24303990298FDF7EE
:102E70002DFB3A46049BFDF795F903910290E089FA
:102E8000FDF74EFB2A463346FDF740FA074604910C
:102E9000208AFDF745FB2A463346FDF737FA2A46D6
:102EA0003346FDF733FA1225ED432A46FDF70EFBB4
:102EB0003A46049BFDF776F92A46FDF707FB0546DF
:102EC0000E46A089FDF72CFB0C4607460E22D24386
:102ED00028463146FDF7FAFA00223C4BFDF762F92D
:102EE0003A462346FDF712FA002204460D461346E1
:102EF000FDF748FB02D100200BB0F0BD2C4E306A2C
:102F0000FDF70EFB0022324BFDF7F7F907460B22C7
:102F10000591D24303990298FDF7D8FA3A46059BEA
:102F2000FDF7EBF900222B4BFDF7F0F922462B467B
:102F3000FDF754FA04460D46B08BFDF7F1FA224630
:102F40002B46FDF7E3F922462B46FDF7DFF91E225B
:102F5000D243FDF7BBFA01910090708BFDF7E0FAC8
:102F600022462B46FDF7D2F90E22D243FDF7AEFAE8
:102F700003910290308BFDF7D3FA06460F46684660
:102F80000FC8FDF70FF932463B46FDF70BF9032258
:102F9000D243FDF79BFA22462B46FDF703F9024682
:102FA0000B460DA0FFF776F90E48FDF726FCBFE6AD
:102FB00000000020340000200000B44054656D3A49
:102FC00025312E31660D0A000040EF400000F03F31
:102FD00000003041006AB84050613A25312E316618
:102FE0000D0A00008813000000000000000000002F
:102FF0000102030406070809030406080C10182040
:103000003000000000010203040000002C30000822
:103010000000002034000000FC220008603000089E
:10302000340000200C0500000C230008B6FF00004F
:103030000000000000000000000000000000000090
:103040000000000000000000000000000000000080
:103050000000000000000000000020000000000050
:04000005080000C12E
:00000001FF
